:100000000C9442070C945F070C945F070C945F07F5
:100010000C945F070C945F070C945F070C945F07C8
:100020000C945F070C945F070C9457230C941323D4
:100030000C94AA240C945F070C945F070C945F0740
:100040000C945F070C945F070C945F070C945F0798
:100050000C945F070C9486240C945F070C945F0744
:100060000C945F070C945F070C945F070C945F0778
:100070000C945F070C945F070C945F070C945F0768
:100080000C945F070C945F070C945F070C945F0758
:100090000C945F070C945F070C945F070C945F0748
:1000A0000C945F070C945F070C945F070631FF09FF
:1000B00074A1010975150026FF00952075088102BD
:1000C0000976150026FF00952075089102C00501EC
:1000D0000902A10185020901A100050919012908E8
:1000E00015002501950875018102050109300931C6
:1000F0001581257F95027508810609381581257FB0
:10010000950175088106050C0A38021581257F9531
:100110000175088106C0C005010980A10185031988
:10012000012AB700150126B700950175108100C09E
:10013000050C0901A101850419012AA00215012657
:10014000A002950175108100C005010906A1018575
:1001500006050719E029E7150025019508750181B5
:10016000020507190029EF1500250195F075018199
:10017000020508190129059505750191029501757A
:10018000039101C00660FF0961A101096215002603
:10019000FF009520750881020963150026FF009570
:1001A0002075089102C005010906A101050719E0A3
:1001B00029E715002501950875018102950175084B
:1001C00081010507190029FF150026FF0095067516
:1001D0000881000508190129059505750191029509
:1001E0000175039101C00000000000000000000044
:1001F00000000000000000000000000000000000FF
:10020000000000000000000000007E0F00D4FFFF8F
:10021000FFC70000007800000000000000002A2B4B
:1002200028000000000000000000000000000000A6
:100230000029000000002C1E34202122243426270F
:10024000252E362D3738271E1F2021222324252630
:100250003333362E37381F0405060708090A0B0CFE
:100260000D0E0F101112131415161718191A1B1C46
:100270001D2F3130232D350405060708090A0B0C04
:100280000D0E0F101112131415161718191A1B1C26
:100290001D2F3130354C44454255473A206469732F
:1002A00061626C65642E0A0044454255473A2065F8
:1002B0006E61626C65642E0A003F00433E2000615F
:1002C00064645F6B65795F6269743A2063616E276D
:1002D00074206164643A20253032580A0064656CE9
:1002E0005F6B65795F6269743A2063616E27742081
:1002F00064656C3A20253032580A004F6E65736889
:100300006F743A206163746976653A2025640A0047
:100310000A002530325820006B6579626F61726483
:100320005F7265706F72743A20005B735D000A0043
:100330002530313662003A200025303258000A72EA
:100340002F63203031323334353637383941424328
:100350004445460A000A0025303258006C65645F47
:100360007461736B3A2000290A002575002F00255F
:1003700075005D280025640020002564002000250C
:10038000640020002564007C0025303258006D6F29
:100390007573656B6579205B62746E7C782079205B
:1003A0007620685D287265702F61636C293A205B46
:1003B000006B65796D61705F636F6E6669672E7241
:1003C00061773A20253032580A2E737761705F6367
:1003D0006F6E74726F6C5F636170736C6F636B3A96
:1003E0002025750A2E636170736C6F636B5F746F89
:1003F0005F636F6E74726F6C3A2025750A2E737787
:1004000061705F6C63746C5F6C6775693A20257509
:100410000A2E737761705F7263746C5F72677569BF
:100420003A2025750A2E737761705F6C616C745F7A
:100430006C6775693A2025750A2E737761705F7253
:10044000616C745F726775693A2025750A2E6E6F4C
:100450005F6775693A2025750A2E737761705F674B
:10046000726176655F6573633A2025750A2E73772E
:1004700061705F6261636B736C6173685F6261631B
:100480006B73706163653A2025750A2E6E6B726F0F
:100490003A2025750A0064656275675F636F6E6652
:1004A00069672E7261773A20253032580A2E656EC0
:1004B00061626C653A2025750A2E6D6174726978E7
:1004C0003A2025750A2E6B6579626F6172643A2055
:1004D00025750A2E6D6F7573653A2025750A0065BE
:1004E00065636F6E6669673A0A64656661756C7408
:1004F0005F6C617965723A2025750A000A092D2022
:100500004D61676963202D0A443A09446562756745
:10051000204D65737361676520546F67676C650A6A
:10052000583A094D61747269782044656275672094
:100530004D6F646520546F67676C65202D2053688C
:100540006F77206B65797072657373657320696E60
:10055000206D617472697820677269640A4B3A0988
:100560004B6579626F6172642044656275672054DF
:100570006F67676C65202D2053686F77206B6579F6
:100580007072657373207265706F72740A4D3A09E8
:100590004465627567204D6F75736520546F67679A
:1005A0006C650A563A0956657273696F6E0A533A5A
:1005B000095374617475730A433A09416374697627
:1005C00061746520436F6E736F6C65204D6F646559
:1005D0000A46312D4631303A0953776974636820F1
:1005E000746F204C6179657220302D392028463196
:1005F00030203D204C30290A302D393A0953776993
:1006000074636820746F204C6179657220302D39D5
:100610000A47524156453A09537769746368207412
:100620006F204C6179657220302028616C7465728E
:100630006E617465290A423A094A756D7020746FBB
:1006400020426F6F746C6F616465720A4553433A60
:10065000094A756D7020746F20426F6F746C6F6102
:100660006465722028616C7465726E617465290A14
:10067000453A095072696E7420454550524F4D20DD
:1006800053657474696E67730A4241434B5350411A
:1006900043453A09436C65617220454550524F4DC0
:1006A0000A4E3A094E4B524F20546F67676C650AE9
:1006B000000A092D20436F6E736F6C65202D0A456B
:1006C00053432F713A09717569740A6D3A096D6F58
:1006D0007573656B65790A000A092D20566572737A
:1006E000696F6E202D0A5649443A203078373635E6
:1006F000342876656E306D7472306E29205049440E
:100700003A2030783030363028302D53697874797B
:1007100029205645523A203078303030310A42553F
:10072000494C443A2020284175672031332032302B
:100730003232290A4F5054494F4E533A204C5546B5
:1007400041204D4F5553454B455920455854524132
:100750004B455920434F4E534F4C4520434F4D4D31
:10076000414E44204E4B524F204C544F2034303990
:10077000360A4743433A20382E332E302041565212
:100780002D4C4942433A20322E302E3020415652D1
:100790005F415243483A20617672350A000A092DBA
:1007A00020537461747573202D0A686F73745F6BC6
:1007B0006579626F6172645F6C65647328293A20A1
:1007C000253032580A6B6579626F6172645F7072AE
:1007D0006F746F636F6C3A20253032580A6B6579FD
:1007E000626F6172645F69646C653A2025303258CB
:1007F0000A6B65796D61705F636F6E6669672E6EF7
:100800006B726F3A20253032580A74696D65725FD9
:1008100072656164333228293A202530386C580AD1
:10082000003F004E4B524F3A206F66660A004E4B17
:10083000524F3A206F6E0A000A6D6F7573653A2049
:100840006F66660A000A6D6F7573653A206F6E0AEF
:10085000000A6B6579626F6172643A206F66660A9E
:10086000000A6B6579626F6172643A206F6E0A00EC
:100870000A6D61747269783A206F66660A000A6DC3
:1008800061747269783A206F6E0A000A6465627555
:10089000673A206F66660A000A64656275673A20E7
:1008A0006F6E0A000A0A4A756D70696E6720746F70
:1008B00020626F6F746C6F616465722E2E2E200043
:1008C000433E2000436C656172696E672045455068
:1008D000524F4D0A00313A0964656C6179282A311A
:1008E000306D73293A2025750A323A09696E7465AC
:1008F0007276616C286D73293A2025750A333A099E
:100900006D61785F73706565643A2025750A343AC5
:100910000974696D655F746F5F6D61783A20257544
:100920000A353A09776865656C5F6D61785F737049
:100930006565643A2025750A363A09776865656CFD
:100940005F74696D655F746F5F6D61783A202575BE
:100950000A00703A097072696E742076616C756570
:10096000730A643A097365742064656661756C7412
:10097000730A75703A092B310A646E3A092D310AEF
:100980006C743A092B31300A72743A092D31300AED
:100990004553432F713A09717569740A0A7370657A
:1009A0006564203D2064656C7461202A206D617847
:1009B0005F7370656564202A2028726570656174B4
:1009C000202F2074696D655F746F5F6D6178290AEF
:1009D00077686572652064656C74613A206375722E
:1009E000736F723D25642C20776865656C3D2564C6
:1009F0000A53656520687474703A2F2F656E2E77E0
:100A0000696B6970656469612E6F72672F77696BB6
:100A1000692F4D6F7573655F6B6579730A004D3E85
:100A200020004D25753A25733E20003F0A003D20E9
:100A300025750A003F0A0064656661756C74730A67
:100A40000025750A003F0A000A092D2056616C75C1
:100A50006573202D0A00710A000A092D204D6F755B
:100A600073656B6579202D0A004C25640A003500FA
:100A70001E001F002000210022002300240025006A
:100A8000260027002A002B0014001A000800150079
:100A900017001C0018000C00120013004C00290065
:100AA00004001600070009000A000B000D000E00EC
:100AB0000F0033003400E1001D001B000600190088
:100AC00005001100100036003700380028003900FA
:100AD000E000E200E30001512C002C000251500024
:100AE000510052004F0035021E021F022002210257
:100AF0002202230224022502260227022A003502AE
:100B00001E021F02200221022202230224022502C9
:100B1000260227024C004C003A003B003C003D00FE
:100B20003E003F002D022E022F0230023102010052
:100B3000400041004200430044004500320264028C
:100B40004A004D0001000100010001000100010008
:100B5000010001000351AB00AA00A900AE0035005E
:100B60001E001F0020002100220023002400250079
:100B7000260027002A0035001E001F00200021004B
:100B80002200230024002500260027004C004C00F2
:100B90003A003B003C003D003E003F002D002E008F
:100BA0002F003000310001004000410042004300AE
:100BB00044004500320064004B004E00010001007B
:100BC0000100010001000351010001000100AB0020
:100BD000AA00A900AE003A003B003C003D003E00E8
:100BE0003F00400041004200430044004500010036
:100BF000005C010001000100010001000100010092
:100C000001000100010001000100010001000100DC
:100C100001000100010001000100010001000100CC
:100C200001000100010001000100010001000100BC
:100C300001000100010001000100010001000100AC
:100C4000010001000100010001000100010001009C
:100C5000010001000100010001000100010001008C
:100C6000010001000100010001000100010001007C
:100C7000010001000100010001000100010001006C
:100C8000010001000100010001000100010001005C
:100C9000010001000100010001000100010001004C
:100CA000010001000100010001000100010001003C
:100CB000010001000100010001000100010001002C
:100CC000010001000100010001000100010001001C
:100CD000010001000100010001000100010001000C
:100CE00001000100010001000100010001000100FC
:100CF00001000100010001000100010001000100EC
:100D000001000100010001000100010001000100DB
:100D100001000100010001000100010001000100CB
:100D200001000100010001000100010001000100BB
:100D300001000100010001000100010001000100AB
:100D4000010001000100010001000100010001009B
:100D5000010001000100010001000100010001008B
:100D6000010001000100010001000100010001007B
:100D7000010001000100010001000100010001006B
:100D8000010001000100010001000100010001005B
:100D9000010001000100010001000100010001004B
:100DA000010001000100010001000100010001003B
:100DB0000100010001005B435D005B445D005B538B
:100DC0005D005B575D005B525D0009027B00040122
:100DD00000A0FA090400000103010100092111012A
:100DE00000012240000705810308000109040100F9
:100DF0000203000000092111010001222200070561
:100E000082032000010705030320000109040200FA
:100E1000010300000009211101000122B6000705AD
:100E200084032000010904030002030000000921DB
:100E3000110100012222000705850320000107059A
:100E40000503200001120100020000000854766032
:100E500000010001020001100330002D0053006961
:100E60000078007400790000001403760065006EBD
:100E70000030006D007400720030006E000000044D
:100E80000309040011241FBECFEFDAE0DEBFCDBF9F
:100E900011E0A0E0B1E0E8E0F5E502C005900D92B8
:100EA000A63CB107D9F722E0A6ECB1E001C01D9243
:100EB000AA3DB207E1F70E94D1240C941A2A0C949F
:100EC0000000FF93EF93E091C601F091C7013097C6
:100ED00009F00995EF91FF910895FC01859180300B
:100EE00011F0EFDFFBCF0895FF27E0E230E247FF8C
:100EF0000CC0419597FF09C0EDE260957095809513
:100F00009095611D711D811D911D27FF02C02195C6
:100F100030E350E2AA27660F771F881F991FAA1F88
:100F2000A41710F0A41B63955A95A9F7AA3008F0EE
:100F3000A95FA05DAF93F3956115710581059105DA
:100F400041F7ED3211F4EF93F395F21718F43F9354
:100F5000F395FBCF8F91B5DFFA95E1F70895E9910D
:100F6000F9918591803021F0853219F0AADFF9CF0F
:100F7000089520E0E89455915532C1F3503311F4AF
:100F8000689455915A3348F4505390F3220F022E2F
:100F9000220F220F200D250FF4CF0EF421958991F9
:100FA0009991533619F3533729F1533559F1BC014F
:100FB00088279927E8945C3621F48991999168945F
:100FC0005591543639F446EF7EF077FF0DC08FEF20
:100FD0009FEF0AC055374AE039F0583540E121F01B
:100FE000523642E009F00895FF93EF937DDFEF91D1
:100FF000FF91B7CFFF93EF93FC0181918030B9F35C
:1010000060DFFBCFFF93EF9368DFF1CFDF93CF93E8
:10101000CDB7DEB72596A3DFCF91DF910895E8ED38
:10102000F0E080818E7F80831092E2001092DA00DF
:101030001092E100A0EEB0E08C9181608C938081F1
:101040008F77808319BCA7EDB0E08C918E7F8C9355
:1010500080818F7E80831092A70208952091E40002
:101060003091E50095E6A9012091EC00822F817076
:1010700020FF06C08091E80080FF06C080E0089550
:101080002091E80022FD1AC08091CC02882389F0CB
:10109000853089F08091EB0085FD0FC02091E40040
:1010A0003091E50042175307F9F29150E1F684E0E0
:1010B000089582E0089583E0089581E00895EF9215
:1010C000FF920F931F93CF937C018B010E942E08F8
:1010D000C82F811117C08091E80085FD0BC0809159
:1010E000E8008E778093E8000E942E08882399F309
:1010F000C82F08C0F70181917F018093F100015052
:10110000110949F78C2FCF911F910F91FF90EF900C
:1011100008958091CE0287FF13C08091E80082FF7E
:1011200006C08091E8008B778093E80004C080912E
:10113000CC028111F2CF08958091CC028823D9F39B
:101140008091E80080FFF8CF8091E8008E77ECCFA7
:10115000982F9093E900242F762F50E0891731F0D3
:101160007091EC002091ED005091F00021FD07C03E
:101170009F5F973071F78093E90081E00895309187
:10118000EB003E7F3093EB003091ED003D7F3093DC
:10119000ED003091EB0031603093EB007093EC0088
:1011A0002093ED005093F0002091EE0027FDE0CF5A
:1011B00080E00895B0E0A0E0E0EEF8E00C948A2929
:1011C000C8EDD0E088818F7E8883E7EDF0E08081F4
:1011D0008160808384E082BF81E08093A702888160
:1011E0008E7F888302EE10E0F80110821092DA0000
:1011F00081EEC82ED12CF601108288818F778883EA
:1012000088818068888388818F7D888319BC10924B
:10121000CC021092CD021092CB021092CA0290EE34
:10122000E92EF12CF70180818B7F8083888181609A
:10123000888342E060E080E00E94A808F601808197
:101240008E7F8083F80180818160808380818860C7
:101250008083F70180818E7F80838881806188838D
:10126000CDB7DEB7E8E00C94A629FC018091D4024A
:101270009091D50286179707A0F06115710529F4A2
:101280009091E8009E779093E80090E061157105D9
:1012900051F4911108C08091E80082FF34C080E0D1
:1012A0000895BC01F2CF8091CC028823C1F1853032
:1012B000C1F18091E80083FD30C08091E80082FD9B
:1012C000EACF8091E80080FFE1CF8091F300209188
:1012D000F200382F6115710519F02830310558F0EA
:1012E00091E02830310509F090E02091E8002E7758
:1012F0002093E800CBCF81918093F1006150710978
:101300002F5F3F4FE7CF8091CC02882341F085309B
:1013100041F08091E80083FFBECF81E0089582E034
:10132000089583E0089508958091A902089587E7BC
:1013300097E7909301088093000888E19AE00FB640
:10134000F894A895809360000FBE90936000FFCF43
:101350009C014FB7F89480919B0290919C02A091C0
:101360009D02B0919E024FBF821B930B08952FB731
:10137000F89480919B0290919C02A0919D02B09163
:101380009E022FBF0895209198023091990228174C
:10139000390771F09093990280939802E091960238
:1013A000F0919702309721F00084F185E02D0995A6
:1013B000089520919402309195022817390771F011
:1013C0009093950280939402E0919602F091970297
:1013D000309721F00680F781E02D09950895E0917E
:1013E0009602F0919702309729F00190F081E02D5C
:1013F0000995089580E0089540918902803F59F44D
:1014000080918A0287FF0DC010928A0241110BC0A1
:101410001092820208C0813F81F480918A021816DE
:101420009CF3442381F080918B0290918C02892B54
:1014300009F05AC0109280020895823F49F447FF94
:10144000F0CF1092890280918A028111ECCFE0CF17
:10145000833F19F41416ACF3E4CF90918B02893FCB
:1014600029F41916F4F610928B02DBCF8A3F19F497
:1014700097FFD7CFF8CF90918C028B3F29F497FF3D
:10148000D0CF10928C02CDCF8C3F19F41916CCF32B
:10149000C8CF9CE0980F953090F4845F990B21E0C1
:1014A00030E0B90102C0660F771F8A95E2F7CB01E1
:1014B000809590918802892380938802B2CF8D3FD6
:1014C00031F4809181028E7F80938102AACF8E3F7A
:1014D00021F4809181028D7FF7CF8F3F09F0A1CF5A
:1014E000809181028B7FF0CF08958091810280FFEF
:1014F0000CC060910D0170E07595679575956795C5
:101500006115710549F1862F089581FF06C060912C
:101510000D0170E075956795F3CF60910D0182FD27
:101520000BC0909180029923A1F060910C018091F1
:101530000D01961738F0682F70E06038710500F3E0
:101540008FE70895899FC001112470E00E945F29F0
:10155000F4CF61E070E0D7CF81E0089580918102FF
:1015600080FF0DC060910F0170E0660F771F60383B
:10157000710570F56115710569F1862F089581FF78
:1015800007C060910F0184E0689FB0011124EFCF84
:1015900082FF04C060910F0188E0F6CF8091820243
:1015A000882399F020910E0160910F018217A0F716
:1015B000869FC001112433E0880F991F3A95E1F707
:1015C000622F70E00E945F29D2CF68E070E0D5CF33
:1015D0008FE7089581E00895803F31F40E94AE0ABC
:1015E000819580938A020895813F19F40E94AE0A82
:1015F000F8CF823F31F40E94AE0A81958093890230
:101600000895833F19F40E94AE0AF8CF893F29F468
:101610000E94750A80938B0208958A3F21F40E94EC
:10162000750A8195F7CF8B3F31F40E94750A819539
:1016300080938C0208958C3F19F40E94750AF8CFAC
:101640009CE0980F953070F4845F990B21E030E0B6
:1016500001C0220F8A95EAF780918802822B80933D
:10166000880208958D3F31F48091810281608093DA
:10167000810208958E3F21F4809181028260F7CF2C
:101680008F3FB9F7809181028460F1CFF894E82F01
:10169000E295EF70F0E031A1282F2F7081E090E00B
:1016A00001C0880F2A95EAF7982F9095932391A36C
:1016B00092A1892B82A37894089590919F0292FF22
:1016C00006C0282F28712830F9F4877F846093FFA3
:1016D00006C0282F28712831F1F4877E846120917B
:1016E000A00220FF06C0382F38713830D9F4877F28
:1016F000816021FF06C0282F28712831D1F4877E10
:10170000816194FD877E0895282F24712430F9F695
:101710008B7F8860DCCF282F2471243101F78B7EEA
:101720008861DDCF382F3171313019F78E7F8860B5
:10173000E0CF282F2171213121F78E7E8861E1CF02
:10174000CF93DF93EC0182389105A9F1D8F581336D
:10175000910509F496C048F58932910509F48AC0CB
:101760008A9709F495C0C11521E5D20708F0BCC0DD
:10177000C11530E5D30708F014C1C83ED10508F003
:101780009CC0C03ED10560F5C83AD10508F087C0BD
:10179000C53AD10508F0FDC0C130D10509F1209747
:1017A000F9F0C430D105E0F440C08533910509F467
:1017B0005AC0C997C1F680919F02837089F0C0EE2C
:1017C000D0E00EC0833E910599F170F4803E910502
:1017D00001F1823E910539F680919F0282FD21C080
:1017E000CE01DF91CF910895863E910561F1873E4C
:1017F000910571F1843E910509F0B5CF8091A00269
:1018000081FFEECF80919F02C7EED0E084FD0DC036
:10181000E7CF80919F0280FD12C19091A00290FFBE
:10182000DFCFC3EED0E084FFDBCFD0E0C0E0D8CF85
:1018300080919F0282FD06C19091A00290FDBFCFD2
:1018400084FFCECFF2CF80919F0283FDDDCFC8CF42
:1018500080919F0283FDF9C09091A00291FFF0CF8B
:10186000C4EED0E0BDCF80919F0285FFB9CFC9E221
:10187000D0E0B6CF80919F0285FFB2CFC5E3D0E024
:10188000AFCF80919F0286FFABCFCAE2D0E0A8CF56
:1018900080919F0286FFA4CFC1E3D0E0A1CFCF3BD0
:1018A000D10518F6C85AD0E0CC0FDD1FCD58DE4F59
:1018B0000990D881C02DD46493CFC11540E2D407DC
:1018C00058F4C11581E0D80708F08ACFC03FD10590
:1018D00008F4ABCFD06584CFC11590E4D90708F4E4
:1018E000A4CFDF70D06A7CCFC11525E5D20700F503
:1018F000C11534E5D30708F08AC0C11543E5D40704
:1019000008F071C0C11582E5D80708F467C0CE01A0
:101910008370992721E030E002C0220F331F8A959F
:10192000E2F7C695C69580E2C89FE001112452C037
:10193000C11599E5D907A8F4C11528E5D20708F023
:101940006BC0C11536E5D30708F06FCF8C2F0E940E
:101950005D0BC82FD0E0DC2FCC27CC27DF71D06205
:101960003FCFC1154AE5D40708F45BC0CE019056BD
:101970008115904208F059CF8D2F8F710E945D0B19
:1019800090E0982F882788279F719C012C2BE901D4
:10199000E6CFC55AD0E0C059DE4FC881D0E0D06450
:1019A0001FCFCE01E4E096958795EA95E1F7837025
:1019B0002C2F26952695237040E2249F9001112418
:1019C000382B8C2F8370C1E0D0E002C0CC0FDD1F1C
:1019D0008A95E2F7C22BD32BDC6802CFDC2FCC2711
:1019E000C16FD06AFDCECE018370992721E030E02F
:1019F00002C0220F331F8A95E2F7C695C69590E282
:101A0000C99FE0011124C22BD32BDA68E9CEDC2F69
:101A1000CC27C46FD06AE4CEDC2FCC27C06FD06A4D
:101A2000DFCE8C2F8F700E945D0B34E0D695C7956A
:101A30003A95E1F7CF709C2FEC01D069D1CEC9E384
:101A4000D0E0CECEC2EED0E0CBCEC6EED0E0C8CE57
:101A500080915C02811110925C02089580959091B2
:101A60005B02982390935B020895809138029091D5
:101A70000702981301C008958F5F8770FACF292F4E
:101A8000953078F58C3068F590E03CE0239F800D30
:101A9000911D1124682F677023E0969587952A95EC
:101AA000E1F7FC01EE0FFF1FE80FF91FE751FE4FB2
:101AB00050E040E080E0219130E0062E02C03695F3
:101AC00027950A94E2F721703327042E01C0220FD4
:101AD0000A94EAF7822B4F5F5F4F4330510559F765
:101AE000089580E00895292F953098F58C3088F579
:101AF00090E03CE0239F800D911D1124282F27703A
:101B000041E001C0440F2A95EAF723E096958795B6
:101B10002A95E1F7FC01EE0FFF1FE80FF91FE751CF
:101B2000FE4F30E020E070E05191DF011197CB01D2
:101B3000022E02C0969587950A94E2F781708195EE
:101B40008527842385278C932F5F3F4F23303105D2
:101B500059F7089581FF02C02E9A08952E9808958E
:101B6000829590E09C01220F331F220F331F2C7CA3
:101B700095958795959587958373282B30E0C901B6
:101B8000880F991F8A7A359527952575822B089598
:101B90009FB7F8941092A5029FBF9091CC02943009
:101BA00009F048C02091E9002F703091EC00932F8C
:101BB000917030FD90E8922B25E02093E900209170
:101BC000EB0020FF34C02091EE0027FF30C02091B1
:101BD000A402222321F02091E80025FF28C01092C2
:101BE000A40226E03091E80035FF14C08093F10094
:101BF0008091E80085FD27C08091E80080FFFCCF40
:101C00008091E8008E778093E8009F709093E900C0
:101C100080E008953091CC02343049F43091EB00EB
:101C200035FD05C0215041F481E08093A4029F70EE
:101C30009093E9008FEF0895EFE9FFE03197F1F716
:101C400000C00000CFCF8FB7F89421E02093A50209
:101C50008FBFDBCF8093A1027093A3026093A20297
:101C60008091CC028430F9F48093E9008FEF909159
:101C7000E800815095FD06C095ED9A95F1F70000BA
:101C80008111F5CF8091E80085FF0DC050E040E064
:101C900063E070E081EA92E00E945F088091E800D2
:101CA0008E778093E8000895BC0184E00E942A0E9C
:101CB0000895BC0183E00E942A0E08959C0184E0EF
:101CC0008093E9009FEF8091E800915085FD06C068
:101CD00085ED8A95F1F700009111F5CF8091E8002C
:101CE00085FF0CC050E040E066E070E0C9010E9452
:101CF0005F088091E8008E778093E8000895CF9385
:101D0000DF93EC01809112018823B1F180919F0251
:101D100087FF32C060E284E08093E9008FEF90910A
:101D2000E800815095FD06C095ED9A95F1F7000009
:101D30008111F5CF8091E80085FF1BC080911201D1
:101D400070E050E040E0811104C050E040E068E005
:101D500070E0CE010E945F088091E8008E7780934A
:101D6000E80080E2FE01AAEAB2E001900D928A95B5
:101D7000E1F7DF91CF91089568E081E0CDCFCF9377
:101D8000DF93CFE6D3E060E0CE010E94D92921960F
:101D9000C11584E0D807B9F7DF91CF9108951F935B
:101DA000CF93DF93122F8730E0F46530D0F44C30BE
:101DB000C0F4C42FD0E0CC0FDD1F98E1699FC00DA7
:101DC000D11D112498E7899FC00DD11D1124632FC7
:101DD000CE0187960E94D929612FCE0188960E9454
:101DE000D929DF91CF911F910895AF92BF92CF92E1
:101DF000DF92EF92FF921F93CF93DF938EE6C82E70
:101E00008AE0D82ED0E07601C0E014C0F50125911B
:101E10003491412F6C2F8D2F0E94CF0E82E0A80E9F
:101E2000B11C1F5F1C3091F788E1E80EF11CCF5FF9
:101E3000C53019F0570110E0E9CFDF5F88E7C80E21
:101E4000D11CD73001F7DF91CF911F91FF90EF9018
:101E5000DF90CF90BF90AF900895CF93C82F6FEFD2
:101E6000811162E283E290E00E94D9296FEFC111F3
:101E700068E084E290E00E94D9296FEFC11163E12C
:101E800085E290E00E94D929CF91089580E00E94D8
:101E90002D0F60E086E290E00E94D9290E94F50EA5
:101EA0000E94BF0E81E00E942D0F08950F931F9393
:101EB000CF93DF93873030F5653020F54C3010F547
:101EC000C42FD0E0CC0FDD1F28E1629FC00DD11DD3
:101ED000112438E7839FC00DD11D1124CE018796B0
:101EE0000E94CB29082F10E0102F0027CE018896E2
:101EF0000E94CB299801282BC901DF91CF911F9116
:101F00000F91089590E080E0F8CF462F873040F49D
:101F1000753030F46C3020F4672F0E94560F08950E
:101F200090E080E00895CF92DF92FF920F931F938D
:101F3000CF93DF936C010091D90280915D02082B51
:101F4000C7E0D0E010E0FC2EC8010C2E02C0959531
:101F500087950A94E2F780FD0CC02197A0F7F12C39
:101F60008F2DDF91CF911F910F91FF90DF90CF9038
:101F70000895B6018C2F0E94850F0E94A00B019737
:101F800061F3EECFCF93DF93EC010E94930FBE017C
:101F90000E94850F0E94A00BDF91CF910895FC0154
:101FA000808191810E94C20F92959F70963091F02E
:101FB00058F4925F9F70923058F4803F19F030F4DB
:101FC000883E30F481E008959A5FF4CF843FD1F3E6
:101FD00080E00895883EB0F3813FD1F7F3CF83E2EC
:101FE00090E00E94CB29823289F484E290E00E9442
:101FF000CB29883059F485E290E00E94CB2991E00A
:10200000833109F090E0892F8170089580E0FCCF42
:10201000CF9384E090E00E94CB29C82F82E290E029
:102020000E94CB29982F8C2FCF91089580910C017D
:102030001F928F9380910D011F928F9380910E01BB
:102040001F928F9380910F011F928F9380911001A7
:102050001F928F93809111011F928F9385ED98E0CD
:102060009F938F930E9406088DB79EB70E960FB66A
:10207000F8949EBF0FBE8DBF0895883228F58E312B
:1020800008F072C08B3041F130F4873009F4CFC0D2
:1020900084E39AE0E0C0833109F45FC08431C1F782
:1020A00086E59AE00E946D0780919302882309F4E7
:1020B000FEC010929302109292021092910210921E
:1020C000900210928F0220C08F3409F4C7C0D8F557
:1020D000893231F38833E1F689E59AE00E946D0791
:1020E0000E9416101F9281E08F931F9288E08F93B9
:1020F00082E599E09F938F930E9406080F900F90BE
:102100000F900F900F900F9020919302222309F4CB
:10211000C9C080918F0290919002009711F483E1E1
:1021200091E09F938F931F922F9382E29AE09F9367
:102130008F930E9406080F900F900F900F900F90B2
:102140000F9081E00895813509F49CC008F49CC08B
:10215000823509F09DCF81E082C088E49AE00E9438
:102160006D070E941610D0CF8D518093930283305B
:1021700009F442C058F48130C1F08230A1F11092CC
:10218000930285E49AE00E946D071BC0853009F434
:1021900045C0D8F1863099F78CE091E09093920297
:1021A000809391028BE591E008C081E191E09093EA
:1021B00092028093910287E191E090939002809344
:1021C0008F0280919302882309F49ECF1F928F93F0
:1021D00081E49AE09F938F930E9406080F900F90DE
:1021E0000F900F9091CF80E191E0909392028093B5
:1021F000910280E291E0E1CF8FE091E09093920232
:10220000809391028CE291E0D8CF8EE091E09093A0
:1022100092028093910289E391E0CFCF8DE091E02B
:10222000909392028093910288E491E0C6CF81E07E
:102230008093110184E1809310018AE080930F0163
:102240008EE180930E0188E080930D0188E28093F7
:102250000C0187E39AE00E946D0756CF8AE0E09177
:102260009102F09192023097D1F02081082E000C5B
:10227000990B820F911D8F3F910541F03CF08FEF3C
:10228000808307C08FEFEBCF86EFE9CF97FFF8CFC2
:10229000108280811F928F938EE29AE09BCF8BE217
:1022A0009AE0D9CF8EE19AE00E946D074ACF80E094
:1022B000089580918E0283FF7EC08EE893E00E9495
:1022C0006D07809188021F928F9389E893E09F9316
:1022D0008F930E94060887E893E00E946D07809123
:1022E0008902282F082E000C330B3F938F9384E82C
:1022F00093E09F938F930E94060882E893E00E94E8
:102300006D0780918A02282F082E000C330B3F9313
:102310008F938FE793E09F938F930E9406088DE73A
:1023200093E00E946D0780918B02282F082E000CED
:10233000330B3F938F938AE793E09F938F930E9491
:10234000060888E793E00E946D0780918C02282F91
:10235000082E000C330B3F938F9385E793E09F93F8
:102360008F930E94060882E793E00E946D07809198
:1023700082021F928F938FE693E09F938F930E9428
:1023800006088DE693E00E946D07809181021F92FE
:102390008F938AE693E09F938F930E94060887E6C7
:1023A00093E00E946D078DB79EB74C960FB6F894D8
:1023B0009EBF0FBE8DBF0E94B7099C0190918902FC
:1023C00080918A02982B21F0309386022093850217
:1023D00090918B0280918C02982B21F03093840293
:1023E00020938302E0919602F0919702309749F092
:1023F00082E0809387020480F581E02D87E892E0F7
:102400000995089590911201992359F190919F0295
:1024100097FF27C0E82FE695E695E695EE3180F424
:10242000F0E0E853FE4F282F277081E090E001C0D4
:10243000880F2A95EAF780959281892382830895EF
:1024400090918E0290FF19C01F928F938DED92E0B4
:102450009F938F930E9406080F900F900F900F90FC
:102460000895EAECF1E09191891303C0DF0111971F
:102470001C9291E0E03DF907B1F7089590911201A7
:10248000992349F190919F0297FF25C0E82FE69587
:10249000E695E695EE3170F4F0E0E853FE4F877074
:1024A00021E030E001C0220F8A95EAF78281822B79
:1024B0008283089590918E0290FF1EC01F928F9389
:1024C0008FEB92E09F938F930E9406080F900F90DE
:1024D0000F900F900895AAECB1E0EFEF90E02D91EE
:1024E000821751F0EF3F19F4211101C0E92F9F5FCE
:1024F0009630A9F7EF3F09F408950E2E000CFF0B5C
:10250000E853FE4FD5CFAAE0B0E0E9E8F2E10C9441
:1025100086298E010F5F1F4F8AE0F80111928A957C
:10252000E9F791EAE92E91E0F92E6801AA24A39433
:10253000B12CF70181917F018F3F09F446C0F894D7
:10254000E82FE295EF70F0E021A18F70A50102C0A5
:10255000440F551F8A95E2F7CA01922F982B91A339
:1025600092A18095892382A3789400C0E6EAF1E0E5
:1025700021E030E0912C812C41914F3F09F481C042
:10258000A42FA295AF70B0E090968C9190E04F7020
:1025900002C0959587954A95E2F780FD72C0C90102
:1025A000882A992A220F331F51E0E23BF50721F7D1
:1025B000F701319780818F3F11F00E94460B80EA2E
:1025C0008A95F1F7F60191828082F2E0CF0ED11C5C
:1025D00046EAE41641E0F40609F0ABCF4AE050E0E9
:1025E000B80181E692E00E940D2AFF24F39400973F
:1025F00009F4F12C892B09F447C08AE0F801A1E61F
:10260000B2E001900D928A95E1F781E0809360023B
:102610000E94B70990935F0280935E0280915E02F0
:1026200090915F020E94A809059790F18091610244
:102630009091620290937702809376028091630278
:102640009091640290937902809378028091650260
:102650009091660290937B0280937A028091670248
:102660009091680290937D0280937C028091690230
:1026700090916A0290937F0280937E021092600292
:1026800007C090E080E08CCF809160028111C6CFBE
:102690008F2D2A96ECE00C94A2290F931F93CF93D1
:1026A000DF9380915B0290915A02892B8093C8013D
:1026B00090915C029923B1F0892B8093C80180919D
:1026C0001201882309F46FC080919F0287FF6BC0BD
:1026D0008EE1EAECF1E090E0815008F066C09111E3
:1026E0000E94280D40E250E06AE372E088EC91E03D
:1026F0000E940D2A892B09F451C080E2E8ECF1E038
:10270000AAE3B2E001900D928A95E1F7E09196027A
:10271000F0919702309709F441C08091120188230B
:1027200059F080919F0287FF07C08091C801809374
:10273000C90186E08093C8010280F381E02D88EC16
:1027400091E0099580918E0282FF28C080FF04C02D
:1027500088E193E00E946D07D0E0C0E002E113E061
:1027600080918E0280FF0EC0FE01E853FE4F8081F3
:102770001F928F931F930F930E9406080F900F9044
:102780000F900F902196C830D10551F780918E029D
:1027900080FF04C080E193E00E946D07DF91CF913C
:1027A0001F910F91089586E094CF2191222309F47F
:1027B00093CF9F5F91CF90E080E00E94D90990E095
:1027C00080E00E94C30910925A020E944D1386E0D5
:1027D000E7E8F2E0DF011D928A95E9F710928202A4
:1027E00010928002109281020E94591108958093E4
:1027F000D9020E94DB1308958091D902982F967018
:10280000963021F488600E94F7130895877FFBCFEC
:1028100021E030E001C0220F8A95EAF720958091EF
:10282000D90282230E94F71308959091390280956E
:10283000892380933902282F277091F4282F082E9E
:10284000000C330B9217130659F09091A00292FFDF
:1028500007C08595859585950E94081410923902C8
:102860000895CF93DF93D82FC091A002C2FB882791
:1028700080F98D1711F1D0FBC2F9C093A0026091CD
:102880009F0284E090E00E94D9296C2F82E290E0C0
:102890000E94D92982E00E94151480918E0280FF47
:1028A0000CC01F92DF938BEF92E09F938F930E9457
:1028B00006080F900F900F900F90DF91CF91089521
:1028C00021E030E001C0220F8A95EAF78091D90219
:1028D000822B0E94F713089580935D020E94DB1300
:1028E0000895882321F00E942E0D0E944D13089513
:1028F000882339F090915B02982B90935B020E94A1
:102900004D130895882309F455C0823879F40E9444
:10291000EF0981FF4FC089E30E943E120E944D13D0
:1029200089E30E9402120E944D130895833859F4DE
:102930000E94EF0980FF3EC083E50E943E120E9484
:102940004D1383E5EECF843859F40E94EF0982FFDE
:1029500031C087E40E943E120E944D1387E4E1CF0C
:102960009CEF980F913AE8F290E2980F983050F46B
:10297000877091E001C0990F8A95EAF7892F0E942C
:102980002E0DD1CF9BE5980F933028F490E080E096
:102990000E94D909089598E5980F973128F490E09E
:1029A00080E00E94C3090895803F20F00E94FC0946
:1029B0000E945911089510925B0280911201EAEC75
:1029C000F1E0882361F080919F0287FF08C08EE1CB
:1029D000DF011D928A95E9F70E94DB13089586E0D6
:1029E000F7CFAAE2B0E0E7EFF4E10C948F298EEC88
:1029F00092E02091F100DC012D93CD01B2E0863D03
:102A00009B07B9F78091CF02833009F472C0B8F404
:102A1000813009F449C0823009F4B3C08091E800E4
:102A200083FF91C28091CE029091CF029A3008F03C
:102A30008AC2E92FF0E0E45EF54D0C9473298A30E8
:102A400009F48EC08B3009F471C0893039F7809158
:102A5000CE02813219F78091D2029091D302009771
:102A600011F00297D9F68091E800877F8093E80003
:102A70008091E80082FF38C09091F3008091F200CD
:102A8000029731F48091F100813011F0863021F409
:102A90008091F1008093A9028091E8008B77809368
:102AA000E8000E948908BACF8091CE02813A09F0ED
:102AB000B5CF8091E800877F8093E8008091D202B3
:102AC0009091D302892B61F460E28AEA92E070E08F
:102AD0000E9435098091E8008B778093E8009ECFB3
:102AE00060E090E080E0F3CF8091CC028111C0CF14
:102AF00095CF8091CE02813A09F090CF8091D20299
:102B00009091D302892B09F089CF8091E800877FCB
:102B10008093E8008091E80080FFFCCF8091120153
:102B20008093F1008091E8008E77B9CF8091CE023A
:102B3000813209F073CF8091D2029091D302892B18
:102B400009F06CCF8091E800877F8093E8000E94B5
:102B500089088091D002809312010E94DB145ECF1D
:102B60008091CE02813209F059CF8091E800877FB1
:102B70008093E8000E9489088091D1028093A80286
:102B80004DCF8091CE02813A09F048CF8091E80084
:102B9000877F8093E8008091E80080FFFCCF8091E0
:102BA000A802BECF803899F0823809F0CCC180915C
:102BB000D2028F70873008F0C6C18093E9008091FF
:102BC000EB0085FB882780F91092E90006C0809110
:102BD000CA029091CB02911182609091E800977F98
:102BE0009093E8008093F1001092F1008091E8004A
:102BF0008E77A5C1882309F493C1823009F0A3C15F
:102C00008091D002811196C18091D2028F702FEFF6
:102C1000280F263008F097C18093E9002091EB003F
:102C200020FF88C1933031F48091EB008062809363
:102C3000EB0080C19091EB0090619093EB0021E05C
:102C400030E001C0220F8A95EAF72093EA00109243
:102C5000EA008091EB008860EACF811174C1109185
:102C6000D0021F778091E3008078812B8093E3006E
:102C70008091E800877F8093E8000E948908809116
:102C8000E80080FFFCCF8091E30080688093E30040
:102C900082E0111183E08093CC0255C180588230CC
:102CA00008F051C12091D0023091D1022C3DE3E0D7
:102CB0003E07A1F583E08A838AE289834FB7F894BF
:102CC000DE01139620E03EE051E2E32FF0E0509366
:102CD0005700E49120FF03C0E295EF703F5FEF7073
:102CE0008E2F90E0EA30C0F0C7968D939D932F5FB2
:102CF000243159F74FBF8091E800877F8093E80027
:102D00006AE270E0CE0101960E9435098091E800E8
:102D10008B778093E80017C1C096E7CF8091D202ED
:102D20009091D302432F55274330510509F44AC0EF
:102D300078F54130510509F47AC08BE790E0EAEC70
:102D4000FDE04230510509F0FEC02091E800277FE8
:102D50002093E8002091D4023091D5028217930786
:102D600008F49C0140E02115310509F065C04111CE
:102D700063C08091E80082FDC9CF8091CC02882396
:102D800029F2853019F28091E80083FFF2CFBECF9F
:102D90004132510509F43CC04232510509F0D3C01B
:102DA0008430910508F0CFC0FC01EE0FFF1FEA54FC
:102DB000FE4F0190F081E02D8E549E4FDC018C91EE
:102DC00090E01AC0332721303105D1F021153105AB
:102DD00061F02230310509F0B6C0E7E5FEE0E4918C
:102DE0008E2F90E0E7E5FEE007C0EFE7FEE0E4911C
:102DF0008E2F90E0EFE7FEE0009709F4A4C0A5CF86
:102E0000E9E6FEE0E4918E2F90E0E9E6FEE0F4CF03
:102E10008430910508F097C0880F991FFC01E25497
:102E2000FE4F0190F081E02D89E090E08ECF82E1AD
:102E300090E0E5E4FEE089CF8091CC02882309F49C
:102E400065CF853009F462CF8091E80083FD5ECFC5
:102E50008091E80082FD8DCF8091E80080FF83CFD4
:102E60009091F3008091F2002115310519F088301E
:102E7000910550F041E0089709F040E08091E800AA
:102E80008E778093E8006FCF44914093F1003196A4
:102E9000215031090196E8CF803809F054C0809163
:102EA000E800877F8093E8008091CD028093F10055
:102EB0009DCE811148C01091D002123008F043C05D
:102EC0008091E800877F8093E8001093CD020E94F4
:102ED0008908112311F084E005C08091E30087FD8B
:102EE000FACF81E08093CC0242E061EC81E00E9465
:102EF000A80842E261EC84E00E94A80842E261EC8A
:102F000082E00E94A80842E260EC83E00E94A808E8
:102F100042E261EC85E00E94A8088091CC0213C0D7
:102F20008091D002813079F481E0933009F080E023
:102F30008093CB021092E9008091E800877F809314
:102F4000E8000E9489088091E80083FF0AC0809110
:102F5000E800877F8093E8008091EB008062809397
:102F6000EB00AA96E3E00C94AB29CF93C82F1F92F5
:102F70008F9389E69AE09F938F930E94060881E0E1
:102F800001C0880FCA95EAF70E946C140E94DB14F6
:102F90000F900F900F900F90CF9108950E94DB1427
:102FA0002FEF84E39CE0215080409040E1F700C087
:102FB000000088E19AE00FB6F894A895809360002D
:102FC0000FBE90936000FFCF68EE7EEF90E080E050
:102FD0000E94F72960E082E090E00E94D92960E039
:102FE00083E090E00E94D92910925D0260E084E0C5
:102FF00090E00E94D92964E082E290E00E94D92901
:1030000060E085E090E00E94D92960E086E090E0F1
:103010000E94D9296FEF87E090E00E94D92940E013
:1030200050E0BA0188E090E00E94EB2960E08DE07A
:1030300090E00E94D92940E050E0BA0188E190E098
:103040000E94EB2960E087E190E00E94D92940E0EE
:1030500050E0BA018CE190E00E94EB2970E060E062
:1030600080E290E00E94F72940E050E0BA0188E158
:1030700090E00E94EB2980E00E942D0F0E94460FF5
:1030800040E050E0BA018FE090E00E94EB2940E080
:1030900050E0BA0183E190E00E94EB290895CF92BD
:1030A000DF92EF92FF921F93CF93DF93EBEFE80F46
:1030B000EF3308F043C1F0E0EA5DF54D0C9473295D
:1030C00083E090E00E94CB291F928F938FED94E0D4
:1030D0009F938F930E94060882E090E00E94CB2984
:1030E00083FB992790F91F929F9382FB992790F970
:1030F0001F929F9381FB992790F91F929F93982F7E
:1031000091701F929F931F928F9386E994E09F93F3
:103110008F930E9406080E94081087FB222720F93F
:103120001F922F9386FB222720F91F922F9385FB56
:10313000222720F91F922F9384FB222720F91F9228
:103140002F9383FB222720F91F922F9382FB2227A4
:1031500020F91F922F9391FB222720F91F922F9382
:10316000292F21701F922F9381FB222720F91F9274
:103170002F93282F21701F922F939F938F9381EB72
:1031800093E09F938F930E9406088DB79EB7889611
:103190000FB6F8949EBF0FBE8DBF81E01CC084ECBB
:1031A00098E00E946D070E94E417F7CF8CEF94E03F
:1031B0000E946D07F2CF80918E02807F80938E02F5
:1031C00081EB96E00E946D0780EC98E00E946D070D
:1031D00081E080938D02DF91CF911F91FF90EF905E
:1031E000DF90CF90089584EA98E00E946D070E94D6
:1031F000DB149FEF24E38CE0915020408040E1F706
:1032000000C000000E94970990918E02892F8E7F46
:1032100090FF816080938E0280FF03C088E998E070
:10322000C7CF8BE898E00E946D0780918E02817F66
:1032300080938E02B2CF90918E02892F8D7F91FF65
:10324000826080938E0281FF08C08EE798E00E9422
:103250006D0780918E028160EBCF80E798E0A8CF68
:1032600090918E02892F8B7F92FF846080938E02D3
:1032700082FF03C081E698E0EACF81E598E098CF2D
:1032800090918E02892F877F93FF886080938E02B2
:1032900083FF03C085E498E0DACF88E398E088CF25
:1032A00088ED96E085CF8FB7F894C0909B02D090C0
:1032B0009C02E0909D02F0909E028FBFC0919F0201
:1032C000C7FBCC27C0F91091A802D09112010E942F
:1032D000EF09FF92EF92DF92CF921F92CF931F924E
:1032E0001F931F92DF931F928F938DE997E09F9317
:1032F0008F930E9406088DB79EB70E960FB6F8946E
:103300009EBF0FBE8DBF49CF0E94DB1490919F02DC
:10331000892F97FB87F9805880939F0287FF03C00E
:103320008EE298E045CF83E298E042CF80E00E94B1
:10333000B51733CF8953FBCF8D51F9CF81E298E098
:103340000E946D0780E047CFCF93C82F8823C9F034
:103350008238C9F40E94EF0981FD13C089E30E94FD
:103360003E120E944D132FEF81EE94E021508040D9
:103370009040E1F700C0000089E30E9402120E9421
:103380004D13CF9108958338A1F40E94EF0980FD79
:10339000F8CF83E50E943E120E944D132FEF81EE7D
:1033A00094E0215080409040E1F700C0000083E5A8
:1033B000E4CF8438A1F40E94EF0982FDE2CF87E4D4
:1033C0000E943E120E944D132FEF81EE94E0215097
:1033D00080409040E1F700C0000087E4CECF8CEF42
:1033E0008C0F813A08F078C080918D028130B9F15C
:1033F000882359F1823009F45CC010928D028091CB
:103400001201882309F459C080919F0287FF55C09B
:10341000EC2FE695E695E695F0E0E853FE4F8281C5
:1034200090E04C2F477021E030E002C0220F331FA4
:103430004A95E2F782239323892B09F449C08C2F04
:103440000E9402120E944D1343C080915B0282329F
:10345000B1F68C2F0E944F18811193CFD0CF80915D
:103460005B028232B1F3C431C9F048F4CB3059F079
:10347000C031C1F089EB92E00E946D0711C0C932E2
:1034800069F0C833B9F781EB96E00E946D078BEBCA
:1034900092E00E946D0781E08170DECF10928D0274
:1034A00080E0FACF82E080938D0288E30E943D1095
:1034B000F2CF8C2F0E943D1064CFEAECF1E080ED5A
:1034C00091E02191C21709F4BACF8E179F07C9F76F
:1034D0008C2F0E943E1253CF80E28C0F883068F40C
:1034E000C77021E030E001C0220FCA95EAF7809151
:1034F0005B02822B80935B0242CFEBE5EC0FE33063
:1035000040F4F0E0E059FE4F808190E00E94D9093C
:1035100038CFE8E5EC0FE73150F4F0E0EE0FFF1F95
:10352000ED58FE4F808191810E94C3092ACFC03F90
:1035300008F427CF8C2F0E94EC0A0E94591121CF4A
:103540001F93CF93DF93182FD0E0C0E0893311F49D
:10355000C0E5D0E0812F0E94A419209739F4812F73
:103560000E948214DF91CF911F9108958FE99FE00F
:103570000197F1F700C000002197EFCF0F931F9341
:10358000CF93DF93C62FD42F022FFC018281882393
:10359000A9F06093D8020E94B7099093D702809354
:1035A000D602C77081E001C0880FCA95EAF70E9471
:1035B0007814DF91CF911F910F9108958091D802D7
:1035C000681332C08091D6029091D7020E94A80958
:1035D000883C910548F510E21D0FCD17B9F080E247
:1035E0008C0F883040F4C77081E001C0880FCA9505
:1035F000EAF70E947114183048F481E09D2F97700B
:1036000001C0880F9A95EAF70E947814802F0E94D3
:10361000A01A183070F6D77081E001C0880FDA95D3
:10362000EAF70E947114C5CFC77081E001C0880F0E
:10363000CA95EAF7F6CFA5E0B0E0E1E2FBE10C9431
:1036400081298C01FC0183819481892B31F0808157
:10365000918189238F3F09F059C52596E1E10C94AA
:103660009D290E94930FF82E682F89819A810E94CC
:10367000730D69817A818F2D0E94850F7C01F8017D
:103680008281882309F408C5970122513F452031E2
:10369000310508F02EC58FEF93E00E94CB298111F0
:1036A00028C0FEEEEF0E5FE6852E53E0952EE1106A
:1036B00032C01C821B82442443944AE0342E74019D
:1036C0008FEFE81AF80AC4010E94CB2989831A8275
:1036D000882379F09FEF980F933058F58A834982B9
:1036E00092E0890E911CC7010E94CB298B83811126
:1036F00021C080913902877009F4AFCFF80182812F
:10370000882309F4AACF8091A00282FFA6CF82E08D
:103710000E941514A2CF811424E0920651F3C40133
:103720000E94CB29811101C0EA943FEF831A930ACA
:10373000BECF4701FE0131967F01F7012081222390
:1037400009F4BDCF213009F047C0918182819130C9
:1037500031F4F2E0EF0EF11C0E94A01A07C0923083
:1037600049F422E0E20EF11C0E94A4193FEFE31A93
:10377000F30AE3CF933031F432E0E30EF11C0E9400
:103780008214F4CF943021F08FEFE81AF80AEECFCC
:1037900092E0E90EF11C30E020E0B7016F5F7F4F4F
:1037A000F70141818053990B8A30910550F02150E7
:1037B0003109E0F28FE99FE00197F1F700C00000C6
:1037C000F6CF329EF001339EF00D11249C012E0F96
:1037D0003F1F842F7B01E1CFE22FF0E0EA5EFD4F37
:1037E0005490822F86958695869590E0FC01EA5F3D
:1037F000FD4F64902770712C022E02C0759467945F
:103800000A94E2F7E1E06E227724FC01EA50FE4FD1
:10381000A490B12C022E02C0B594A7940A94E2F7AA
:10382000F1E0AF22BB24FC01EA51FE4FC490D12C41
:1038300002C0D594C7942A95E2F721E0C222DD2484
:103840006114710419F081EE0E94A419A114B1044D
:1038500019F086EE0E94A419852D0E94A01AA114C9
:10386000B10419F086EE0E9482146114710419F0FB
:1038700081EE0E948214C114D10409F477CF8CE246
:103880006BCF81E00E94601403C081E00E940814A5
:103890000E94FC132ECF82E0F9CF95EFE9169CE54C
:1038A000F90609F46CC008F466C027E245EE66EE3E
:1038B000F6EFEF16FCE5FF0609F417C4882309F4B8
:1038C00036C41092D80223E0E2162DE5F20608F085
:1038D0005DC03AEFE3163CE5F30630F4C7018250D1
:1038E0009C45449708F05EC00E9408109093A00287
:1038F00080939F02E1E1EE16ECE5FE0609F436C185
:1039000008F0A4C029E0E2162CE5F20609F41CC177
:1039100008F06DC085E0E8168CE5F80609F408C1EA
:1039200008F056C0E3E0EE16ECE5FE0609F4F6C03A
:1039300008F0FAC080919F02816022E0E2162CE537
:10394000F20609F4EEC060919F02F090A00284E0BC
:1039500090E00E94D9296F2D82E290E00E94D9293F
:103960000E94DB14C6CE27E245EE65EEBEC326E21A
:1039700041EE60EEBAC327E245EE64EEB6C326E23E
:1039800041EE62EEB2C328E241E0EFCF81E6E816F5
:103990008DE5F80609F4A8CF95EAE9169DE5F90644
:1039A00009F4A2CF36E1E3163CE5F30609F0CDC3F6
:1039B00080915B028A7A91E009F490E09093E801AB
:1039C000811102C189E20E943E120E944D1391CEE4
:1039D00080919F02806237E0E3163CE5F30609F42C
:1039E000A0C008F4ADC080919F0280649AC080910D
:1039F0009F028B7F9DE0E9169CE5F90609F491C0D2
:103A0000B0F480919F028E7FFBE0EF16FCE5FF068D
:103A100009F487C080919F028C602CE0E2162CE5AF
:103A2000F20608F47EC080919F028D7F7AC080915B
:103A30009F028F7E3FE0E3163CE5F30609F471C078
:103A400008F488C080919F028F7D6BC09DEFE916BE
:103A50009CE5F90609F486C078F5F5E1EF16FCE57A
:103A6000FF0609F491C0A0F480919F02837F33E1A7
:103A7000E3163CE5F30609F454C008F47BC00E9449
:103A8000DB1490919F02892F97FB87F9805849C0DA
:103A90009BEFE9169CE5F90609F44EC008F05EC0FC
:103AA0008091A0028160FAEFEF16FCE5FF0609F0B5
:103AB0004ACF8093A00247CF21E0E2162DE5F2061F
:103AC00009F46EC0B8F48FEFE8168CE5F80609F437
:103AD00057C08091A0028360E1149DE5F90648F388
:103AE0008091A002982F909591708E7F892B90FBEA
:103AF00081F9DFCFE1E6EE16EDE5FE0609F456C0EA
:103B0000F5EAEF16FDE5FF0609F457C022E0E216DC
:103B10002DE5F20609F017CF60E043C080919F02C7
:103B2000826080939F020FCF80919F028460F9CFC3
:103B300080919F028860F5CF8091A0028260B9CF0A
:103B400080919F028061EDCF0E94DB1480919F02E3
:103B50008068E7CF80919F02877FE3CF8091A002AA
:103B60008E7FA7CF8091A0028D7FA3CF80919F02EF
:103B70008F7BD7CF0E94DB1480919F028F77D1CFAC
:103B80008091A0028C7F95CF80919F0282FB992724
:103B900090F921E0922790FB82F990FB83F9C1CF45
:103BA00061E08EE090E00E94D929CDCE90919F02F5
:103BB000892F8F7E94FF8061B4CF90919F02892FCF
:103BC0008E7F90FF8160ADCF85E3FDCE85E3BAC2E5
:103BD00090918E02892F8E7F90FF816080938E025C
:103BE00080FF05C088EA92E00E946D0782CD86E9D9
:103BF00092E0FACF0E94E4170E94CE178091A002B3
:103C000082FB882780F991E089270E943114F8010E
:103C10008281E080F180882309F445C0C7010E94B9
:103C2000930FD82E682FC7010E94730DB7018D2DF9
:103C30000E94850F0E94A00B7C01882EF801D28083
:103C4000B580B2943FE0B322809139028770C1F011
:103C5000AD2CDD20B1F08F2D807F803421F080E20B
:103C60008E0D883068F08091A00282FF09C082E04A
:103C70000E941514809139028770AA24A39481119F
:103C8000A12C9F2C92942FE09222FBE0F91508F4CE
:103C900079C0E92DF0E0EB59F54D0C94732981E0E2
:103CA000B4CF80E0B2CFC7010E943F0DD82EBECF67
:103CB0002F2D2F70C22E8F2D807F19F0C29490EF80
:103CC000C922DD20B9F0CC2069F080E28E0D883069
:103CD00010F0811009C080915B02C82AC0925B027B
:103CE0000E944D138E2D4CC080915A02C82AC0925A
:103CF0005A02F6CF8E2D0E948214CC2009F442C0C5
:103D000080E28E0D883010F0811004C08C2D0E944E
:103D10002E0D06C0C09480915A02C822C0925A0249
:103D20000E944D132FC03F2D3F70C32E8F2D807FDB
:103D3000803219F0C29480EFC822882089F081E097
:103D4000881609F46AC0DD2009F474C0BB2009F4A8
:103D50006AC0F801858180FFC5CF8F70858363C0FD
:103D60002091A00222FD37C0DD2079F1CC2039F06E
:103D700080915B02C82AC0925B020E944D1380E0D2
:103D80000E94A419292D2850330B2430310520F42A
:103D90000E94EF090E94AA0DAA2009F45ECC80912E
:103DA000390280FD5ACCF80112828595859585955A
:103DB0000E946014C8010E941B1B809139028595E6
:103DC000859585950E94081448CC80E00E94821455
:103DD000CC20C1F29BCFDD2099F090915C028C2D1C
:103DE000892BB11003C00E947814CCCFE1E0BE1241
:103DF000FACF22FFC7CF981729F280935C02C2CF77
:103E0000B11006C00E94280D8C2D0E947114BACFEB
:103E1000F1E0BF1609F4B6CFF5CFDD2031F025E093
:103E20002B1508F4AFCF8C2DDECF34E03B1508F412
:103E3000A9CFEACFBB2041F3F9E38F1209C02FEFDE
:103E400037EE83E0215030408040E1F700C00000B1
:103E50008E2D0E94821496CF8F2D86958695837025
:103E600061F0813009F08ECFC7019370D11002C08C
:103E700090E080E00E94C30985CFC7019370D11004
